:0200000480007A
:10000000971000009380000137F1F11113012122B4
:1000100023A020009712000093821200B74C33F304
:10002000938C4C4FA3AF92FF171400001304F4FEFF
:10003000B7FFF555938F6F66A320F4019715000065
:100040009385057E379677F71306868F23A0C580A4
:10005000170700001307177DB71709999387A7AAF9
:10006000A32FF77E97180000938848FC37D9BB0B65
:100070001309C9C0B7190DDD9389E9EE370AFF0FDF
:10008000130A0A0F23AE28FF23A0380123A2480138
:10009000171B0000130B0BFA375034121300806744
:1000A00023200B00971A0000938ACAF5B739221152
:1000B0009389493483AB0A0023A03B01971B0000BE
:1000C000938B8BF4171C0000130C4CF783AC0B00C4
:1000D00023209C01171D0000130D8DF6B73C5476AC
:1000E000938C0C2123209D01930C0000171E00000F
:1000F000130E4EF5B7DDAB89938DFDDE2320BE01D7
:10010000130ECEFF971E0000938E0EF4B76D72147F
:10011000938D6D8323A0BE0103AF0E0023A2EE01D9
:10012000971000009380C0F23751389613011120C8
:10013000B75181259381319623A0200023A0300060
:1001400017150000130505ED97150000938585F040
:10015000370610F01306C6F26306B5028326C50003
:100160002320D600832685002320D6008326450041
:100170002320D600832605002320D6001305050181
:100180006FF09FFD370510F0130505F223200500E1
:04019000000000006B
:1010000034100080F0DEBC9A0000000000000000F8
:10101000FFFFFFFFFFFFFFFFFFFFFFFFFFFFFFFFE0
:10102000FFFFFFFFFFFFFFFFFFFFFFFFFFFFFFFFD0
:10103000FFFFFFFFFFFFFFFFFFFFFFFFFFFFFFFFC0
:10104000FFFFFFFFFFFFFFFFFFFFFFFFFFFFFFFFB0
:040000058000000077
:00000001FF
